:100000000C9422050C945A050C945A050C945A052C
:100010000C945A050C945A050C945A050C945A05E4
:100020000C945A050C945A050C946A220C94AC2139
:100030000C94891A0C945A050C945A050C945A0580
:100040000C945A050C945A050C945A050C945A05B4
:100050000C945A050C943C1A0C945A050C945A05AD
:100060000C945A050C945A050C945A050C945A0594
:100070000C945A050C945A050C945A050C945A0584
:100080000C945A050C945A050C945A050C945A0574
:100090000C945A050C945A050C945A050C945A0564
:1000A0000C945A050C945A050C945A05590B5C0B88
:1000B0008F0BA20BA80BB30BB60BB60BB60BDF0C5A
:1000C000DF0C2A0C2C0C310C570C7A0C7D0C800C9C
:1000D000A50CC50CD00CC60E3A0FCE0E980E9C0E79
:1000E000D20E9F0ED50EE00EAA0E300FAE0EE40E0D
:1000F000B20EE80E120FB60EEC0E1C0FBC0EF20E76
:10010000FC0EA30ED90EA60EDC0EC10EF70E080FC4
:10011000280F2A0F940ECA0E430F630F690F550E56
:100120005D0F6F0F750F7B0FC60F940F990F9E0F0A
:10013000A30FA80FAD0FB20FB70FBC0FC10FF30F76
:10014000F60FC60F940F990F9E0FA30FA80FAD0FB8
:10015000B20FB70FBC0FC10FDA10DA100D110D116D
:100160008C11AA11AB12AB12AF112312341234123C
:10017000B71FDE1F9421DE1F94212A204D209421D9
:100180004321532193276D27B027B327B82742284F
:10019000452848286565636F6E6669675F7570649A
:1001A0006174655F7267625F6D61747269785F64C4
:1001B000656661756C740A007267625F6D61747266
:1001C00069785F636F6E6669672E666C616773201E
:1001D0003D2025640A007267625F6D617472697800
:1001E0005F636F6E6669672E7370656564203D207E
:1001F00025640A007267625F6D61747269785F637B
:100200006F6E6669672E6873762E76203D202564B2
:100210000A007267625F6D61747269785F636F6E06
:100220006669672E6873762E73203D2025640A0068
:100230007267625F6D61747269785F636F6E666921
:10024000672E6873762E68203D2025640A00726749
:10025000625F6D61747269785F636F6E6669672E45
:100260006D6F6465203D2025640A007267625F6DD2
:1002700061747269785F636F6E6669672E656E611F
:10028000626C65203D2025640A007267625F6D61C3
:10029000747269785F636F6E666967204545505276
:1002A0004F4D0A007267625F6D61747269785F69B1
:1002B0006E69745F64726976657273207267625FDB
:1002C0006D61747269785F636F6E6669672E6D6FBA
:1002D0006465203D20302E20577269746520646566
:1002E0006661756C742076616C75657320746F201F
:1002F000454550524F4D2E0A0073757370656E64FC
:10030000696E67206B6579626F6172640D0A000A1D
:100310000025303862003A200025303258000A7239
:100320002F632030313233343536370A006C656440
:100330005F7461736B3A20253032580A0000000068
:1003400000000000000000000000000000000000AD
:10035000000000000000000000000000000000009D
:10036000007E0F00D4FFFFFFC700000078000000F0
:1003700000000000002A2B28000000000000000000
:10038000000000000000000029000000002C1E34C6
:1003900020212224342627252E362D3738271E1FCC
:1003A000202122232425263333362E37381F0405F7
:1003B000060708090A0B0C0D0E0F10111213141565
:1003C000161718191A1B1C1D2F3130232D35040543
:1003D000060708090A0B0C0D0E0F10111213141545
:1003E000161718191A1B1C1D2F3130354C44454265
:1003F00055473A2064697361626C65642E0A004453
:10040000454255473A20656E61626C65642E0A006C
:100410004F6E6573686F743A206163746976653AEC
:100420002025640A000000150008000C00180000D8
:1004300000000014001A0017000A00120013000048
:10044000000000090007000E000D0000000000047D
:10045000001600050028000F0033000000000019FE
:1004600000060036001000000000001D001B001CEC
:10047000000B0037003800000000002900E100E513
:10048000004C000000AE002B00E00011002C0034F6
:10049000002A00000000000100010001000100002E
:1004A0000000000100010001000100010001000046
:1004B0000000000100010001000100000000000137
:1004C0000001000100010001000100000000000126
:1004D0000001000100010000000000010001000116
:1004E0000001000100010000000000010001000106
:1004F00000010000000100010001000100010001F5
:1005000000010000000000010001000100010000E6
:1005100000000001000100010001000100010000D5
:1005200000000001000100010001000000000001C6
:1005300000010001000100010001000000000001B5
:1005400000010001000100000000000100010001A5
:100550000001000100010000000000010001000195
:100560000001000000010001000100010001000184
:100570000001000000000001000100010001000076
:100580000000000100010001000100010001000065
:100590000000000100010001000100000000000156
:1005A0000001000100010001000100000000000145
:1005B0000001000100010000000000010001000135
:1005C0000001000100010000000000010001000125
:1005D0000001000000010001000100010001000114
:1005E0000001000000A900AA00AB00AC0027782899
:1005F0007850004F00290A002575002F002575004E
:100600005D2800256400200025640020002564008A
:1006100020002564007C0025303258006D6F757312
:10062000656B6579205B62746E7C7820792076201A
:10063000685D287265702F61636C293A205B0061E8
:1006400064645F6B65795F6269743A2063616E27E9
:1006500074206164643A20253032580A0064656C65
:100660005F6B65795F6269743A2063616E277420FD
:1006700064656C3A20253032580A000631FF09744F
:10068000A1010975150026FF00952075088102C09B
:1006900005010902A10185020901A100050919014D
:1006A0002908150025019508750181020501093009
:1006B00009311581257F9502750881060938158154
:1006C000257F950175088106050C0A3802158125DC
:1006D0007F950175088106C0C005010980A10185CB
:1006E0000319012AB700150126B70095017510817D
:1006F00000C0050C0901A101850419012AA00215F9
:100700000126A002950175108100C005010906A10E
:10071000018506050719E029E715002501950875EB
:100720000181020507190029EF1500250195F075D3
:1007300001810205081901290595057501910295A8
:100740000175039101C00660FF0961A101096215ED
:100750000026FF009520750881020963150026FF19
:1007600000952075089102C005010906A101050741
:1007700019E029E715002501950875018102950109
:10078000750881010507190029FF150026FF00954E
:100790000675088100050819012905150025019530
:1007A0000575019102950175039101C05B435D00E0
:1007B0005B445D005B535D005B575D005B525D0019
:1007C00009027400040100A0FA09040000010301F9
:1007D00001000921110100012244000705810308DD
:1007E00000010904010002030000000921110100B9
:1007F00001222200070582032000010705030320D0
:100800000001090402000103000000092111010098
:100810000122B6000705840320000109040300013A
:1008200003000000092111010001221500070585C0
:10083000032000011201000200000008042000CB88
:100840000001010200011803730070006C006100D8
:10085000790074006F00720061006900640000009C
:100860000C0346007200650079006100000004037B
:10087000090400010101010101010101020202025A
:10088000020202020203030303030303030404043A
:100890000404040405050505050606060606070703
:1008A00007070708080808090909090A0A0A0B0BBB
:1008B0000B0C0C0C0D0D0D0E0E0E0F0F0F1010115A
:1008C00011111212131314141515161617171818E0
:1008D00019191A1A1B1B1C1D1D1E1E1F2020212248
:1008E00022232424252626272829292A2B2C2D2D8E
:1008F0002E2F30313232333435363738393A3B3CAB
:100900003D3E3F404142434445464748494A4C4D9D
:100910004E4F50515354555658595A5B5D5E5F6166
:100920006264656668696B6C6D6F707273757778F9
:100930007A7B7D7E8082838587888A8C8E8F919357
:100940009596989A9C9EA0A2A3A5A7A9ABADAFB17E
:10095000B3B5B7BABCBEC0C2C4C6C9CBCDCFD1D463
:10096000D6D8DBDDDFE2E4E7E9EBEEF0F3F5F8FA09
:10097000FDFF726762206D617472697820746F6721
:10098000676C65205B25735D3A207267625F6D61FD
:10099000747269785F636F6E6669672E656E6162F7
:1009A0006C65203D2025750A00726762206D6174B8
:1009B000726978206D6F6465205B25735D3A202530
:1009C000750A00726762206D6174726978207365C0
:1009D0007420687376205B25735D3A2025752C257D
:1009E000752C25750A00726762206D6174726978D2
:1009F00020736574207370656564205B25735D3AB0
:100A00002025750A000A002530325820006E6B72CE
:100A10006F5F7265706F72743A2025303258207C97
:100A200020000A002530325820006B6579626F6122
:100A300072645F7265706F72743A2025303258208C
:100A40007C20000011241FBECFEFDAE0DEBFCDBF57
:100A500004B603FE18C080915E0390915F03A091DD
:100A60006003B09161038730904BA740B04B59F4BD
:100A700010925E0310925F03109260031092610364
:100A8000E0E0F8E3099512E0A0E0B1E0E2E2FDE584
:100A900002C005900D92A430B107D9F723E0A4E07D
:100AA000B2E001C01D92AE35B207E1F70E940A061E
:100AB0000C948F2E0C940000FF93EF93E0910402AE
:100AC000F0910502309709F00995EF91FF91089593
:100AD000FC018591803011F0EFDFFBCF0895FF27F7
:100AE000E0E230E247FF0CC0419597FF09C0EDE21C
:100AF0006095709580959095611D711D811D911D6A
:100B000027FF02C0219530E350E2AA27660F771F26
:100B1000881F991FAA1FA41710F0A41B63955A954C
:100B2000A9F7AA3008F0A95FA05DAF93F39561150E
:100B300071058105910541F7ED3211F4EF93F395BD
:100B4000F21718F43F93F395FBCF8F91B5DFFA9529
:100B5000E1F70895E991F9918591803021F085328E
:100B600019F0AADFF9CF089520E0E89455915532A5
:100B7000C1F3503311F4689455915A3348F45053EB
:100B800090F3220F022E220F220F200D250FF4CFFB
:100B90000EF4219589919991533619F3533729F120
:100BA000533559F1BC0188279927E8945C3621F424
:100BB0008991999168945591543639F446EF7EF0B5
:100BC00077FF0DC08FEF9FEF0AC055374AE039F02D
:100BD000583540E121F0523642E009F00895FF9384
:100BE000EF937DDFEF91FF91B7CFFF93EF93FC0180
:100BF00081918030B9F360DFFBCFFF93EF9368DF23
:100C0000F1CFDF93CF93CDB7DEB72596A3DFCF919A
:100C1000DF910895A3E3B0E0E0E1F6E00C944B2E01
:100C200085B7806885BF85B7806885BF84B7877FB3
:100C300084BF0FB6F894A895809160008861809376
:100C40006000109260000FBE90E080E80FB6F8944C
:100C500080936100909361000FBE81E080930D014D
:100C600087E798E190930502809304020E94F021A7
:100C70000E940F228091E20084608093E2007894C9
:100C8000809115038823A1F01091E9001F709091C5
:100C9000EC00892F817090FD80E8182B1092E900FC
:100CA0008091E80083FD0E94D01E1F701093E90020
:100CB00082E084BD93E095BD9AEF97BD80936E006E
:100CC0000E94B41B811102C00E94481E88E0EBEA1A
:100CD000F2E0DF011D928A95E9F781E080931A0224
:100CE00060E080E00E94951E61E080E00E94951E19
:100CF000EFE8F1E03197F1F700C0000010E08091DB
:100D00001A02181790F460E0812F0E94861E082FA7
:100D100061E0812F0E94861EE12FF0E0E75EFD4F2B
:100D2000880F082B00831F5FEACF09E111E041E241
:100D3000E42E41E0F42ED8018D918D018F3F11F00A
:100D40000E948F29E016F106B1F701E211E0F801E7
:100D500081918F018F3F11F00E948F29F1E00832BD
:100D60001F07A9F788E0EDE1F2E0DF01282F1D92CF
:100D70002A95E9F7E6E0F2E0DF011D928A95E9F7AE
:100D800080E090E00E94D02D853E9E4F21F40E948D
:100D9000B41B811163C065EE7EEF80E090E00E949D
:100DA000042E60E082E090E00E94E62D81E08093D6
:100DB0000E0261E083E090E00E94E62D60E074E1C5
:100DC00084E090E00E94042E60E086E090E00E94C3
:100DD000E62D60E087E090E00E94E62D40E050E0E4
:100DE000BA0188E090E00E94F82D60E083E290E094
:100DF0000E94E62D60E08CE090E00E94E62D60E02D
:100E00008DE090E00E94E62D19821A821B821C82DE
:100E10001D821E821F82188648E050E067E170E064
:100E2000CE0101960E94D62D40E050E0BA018FE13C
:100E300090E00E94F82D80E00E94951B0E94481EC1
:100E400040E050E0BA018FE090E00E94F82D40E0D1
:100E500050E0BA0183E190E00E94F82D82E090E03A
:100E60000E94C82D8093FF0284E090E00E94D02D64
:100E700090930103809300030E94A629EFEFF6E709
:100E800021E0E150F0402040E1F700C000000E9466
:100E9000A62980911E0280FF08C06FEF7FEF80E0DF
:100EA00090E00E94042E0E94181A83E090E00E94B5
:100EB000C82D0E947F160E94751881E0809323033D
:100EC00048E050E067E170E086E593E00E94B82DCD
:100ED00010922303809156038C7FB9F58091FF0215
:100EE00080FF08C084EA92E09F938F930E940106DE
:100EF0000F900F908091FF0280FF08C084E991E07D
:100F00009F938F930E9401060F900F9089E080932A
:100F100056038091160190911701A09118018093BA
:100F2000570390935803A093590382E380935A0385
:100F30008FEF80935B0348E050E067E170E086E567
:100F400093E00E94D62D109223038091FF0280FF30
:100F500008C08AE892E09F938F930E9401060F9049
:100F60000F908091FF0280FF0FC080915603837025
:100F70001F928F938BE692E09F938F930E940106BE
:100F80000F900F900F900F908091FF0280FF10C084
:100F900080915603869586951F928F938EE492E0FA
:100FA0009F938F930E9401060F900F900F900F90C8
:100FB0008091FF0280FF0EC0809157031F928F9394
:100FC00080E392E09F938F930E9401060F900F9011
:100FD0000F900F908091FF0280FF0EC08091580308
:100FE0001F928F9382E192E09F938F930E9401065C
:100FF0000F900F900F900F908091FF0280FF0EC016
:10100000809159031F928F9384EF91E09F938F9368
:101010000E9401060F900F900F900F908091FF0299
:1010200080FF0EC080915A031F928F9386ED91E04E
:101030009F938F930E9401060F900F900F900F9037
:101040008091FF0280FF0EC080915B031F928F93FF
:1010500088EB91E09F938F930E9401060F900F9071
:101060000F900F9080E091E09093FC028093FB0240
:1010700096E1292E93E0392E21E1422E23E0522ED3
:101080003FE0632E33E0732E8E010F5F1F4F809180
:101090001503853009F051C08091FF0280FF08C020
:1010A00089EF92E09F938F930E9401060F900F901B
:1010B000A0E4DA2EB0E1FB2E82E1E82E8091150348
:1010C000853009F036C080911503843029F10E94E3
:1010D000C6261092020388E190E00FB6F894A89516
:1010E000809360000FBED092600083B7817F8460E0
:1010F00083BF83B7816083BF7894889583B78E7FE1
:1011000083BF0FB6F894A8958091600088618093A2
:101110006000109260000FBE0E94A629EDE1F2E08F
:10112000819181114BC1A5E2B2E0AE17BF07C1F7B3
:10113000C5CF0E9482160E94831B0E94A629E0E16F
:10114000CE2EE2E0DE2EFDE1AF2EF2E0BF2E28E152
:1011500032E0D501F60191918D9189272E173F0735
:1011600019F08823C1F305C0811103C00E948D2BA3
:1011700070C08091FF0281FD02C0F12C36C08EE16B
:1011800093E09F938F930E9401060F900F907DE153
:10119000872E72E0972EE12CF12CFF92EF92E9E17D
:1011A000F3E0FF93EF930E9401063F922F920E947B
:1011B0000106D4018D914D010E948C2C1F928F93BA
:1011C0005F924F920E9401067F926F920E940106E9
:1011D000BFEFEB1AFB0A0FB6F894DEBF0FBECDBF10
:1011E000F8E0EF16F104C9F6C8CFD5018D905D0186
:1011F000F601808188258BAB882311F1E12C99249D
:1012000093948BA98921A9F0EDA6FEA60E947D1AD0
:1012100098AB8FA7F1E0F9AB91E0892D882109F413
:1012200090E09AAB4DA55EA56FA578A989A90E940B
:10123000C32CE394990C27E0E212E3CFD6018C9201
:10124000F394BFEFCB1ADB0AE8E0FE12CECF0E9488
:10125000711A0E94C62680911B02882351F01092B9
:101260001B028091AD028093AE028091AB0280930D
:10127000AC02B12C64E0C62ED12C80911A02B816B3
:1012800008F041C061E08B2D0E94861EF82E60E0C0
:101290008B2D0E94861EEF2DEE0F8E2B2B2D30E016
:1012A000D901A75EBD4FEC914E2F437050E0682FDF
:1012B00070E04617570729F1EE0FEE0FE82BEC937D
:1012C000EF70F0E0E85DFE4FC901885E9D4F7C0144
:1012D000A080DC018C91A80EAC92B3E0BA1514F496
:1012E00060E004C0EDEFAE1624F461E08B2D0E94A7
:1012F000AB1E8A2DAA0C990BB6010E942A2ED7018B
:101300008C93B394BACF90E02CEFA22E33E0B32E9F
:10131000CC24C3944DEFD42E52E0E52E8091AE0242
:101320002091AD02281709F464C0E82FF0E0E155E0
:10133000FD4F908197FB992490F89F77F92E8F5F4E
:1013400083708093AE028091AC028F5F8093AC0279
:10135000992041F00E947D1AF9A2DAA29CA38BA3E6
:10136000EDA207C00E947D1AF9A2AAA29CA38BA39A
:10137000BDA2CEA249A15AA16BA17CA18DA19EA123
:101380000E94C32C992041F00E947D1AFFA2D8A68A
:101390009AA789A7EBA607C00E947D1AFFA2A8A65C
:1013A0009AA789A7BBA61CA64FA158A569A57AA58F
:1013B0008BA59CA50E94C32C91E0B0CF8091140313
:1013C000882309F47BCEF9BCE9BC09B400FEFDCF4B
:1013D0008091D8008F7D8093D8008091E00082605A
:1013E0008093E0008091E00081FDFCCF0E94821696
:1013F00065CE91110E94711A86E0E0EFF2E0D8010B
:1014000001900D928A95E1F7A090F102E090F2022E
:10141000F090F302C090F402D090F5021092F20224
:101420001092F3021092F4021092F502E11003C040
:10143000FF2009F447C08091EE029091EF020E94D4
:10144000621A9C019091EB02992309F4CAC22531DA
:101450003105C0F19F3F19F09F5F9093EB02EE20A2
:1014600061F00E94371D1E1414F491E001C09FEF3B
:10147000899F802D11248093F202FF2061F00E9449
:10148000371D1F1414F09FEF01C091E0899F802D3C
:1014900011248093F3028091F202882399F0B09096
:1014A000F302BB2079F00E94571D811101C081E039
:1014B0008093F2028B2D0E94571D811101C081E0A3
:1014C0008093F302C11003C0DD2009F447C080916E
:1014D000EC029091ED020E94621A9C019091E90247
:1014E000992309F483C221353105C0F19F3F19F0DA
:1014F0009F5F9093E902CC2061F00E94151D1C149F
:1015000014F491E001C09FEF899F802D11248093F6
:10151000F402DD2061F00E94151D1D1414F09FEFF0
:1015200001C091E0899F802D11248093F502809164
:10153000F402882399F0B090F502BB2079F00E9464
:10154000571D811101C081E08093F4028B2D0E9410
:10155000571D811101C081E08093F5028091F10255
:101560008A111AC08091F202882311F08E1114C0E2
:101570008091F302882311F0F8120EC08091F502D9
:10158000882311F08D1108C09091F402992331F055
:1015900081E09C1104C002C081E001C080E080FDB8
:1015A00015C08091F20281110FC08091F302811168
:1015B0000BC08091F402811107C081E09091F50287
:1015C000911103C080E001C081E080FD0E94511CA8
:1015D000AA82EB82FC82CD82DE8286E0F801A0EF57
:1015E000B2E001900D928A95E1F70E94831BF82EDC
:1015F00080911C02F816B1F0F0921C020E94711A40
:101600008091FF0282FF0EC080FF0CC01F92FF92EC
:101610008DE293E09F938F930E9401060F900F90AD
:101620000F900F9080911503843009F030CD83E046
:101630008093E9008091E80082FF29CD8091E80045
:1016400085FF21C00E94B82381111BC080E2E82ED3
:10165000F12C680109C08091F100F60181936F01BE
:10166000F1E0EF1AF10869F08091E80085FDF3CF11
:101670008091E8008B778093E8000E94B82388234C
:1016800099F391E001C090E08091E8008B7780931E
:10169000E800992309F4FBCC2981822F90E0FC011A
:1016A0003197E531F10508F08AC1EA5AFF4F0C94F1
:1016B0003E2E1A828CE0D3C08A81823009F488C120
:1016C00050F4813009F07BC10E94711A9B838C8396
:1016D0007D836E8376C1833041F0843009F06FC121
:1016E0001B821C821D821E826CC16B81DE011496DE
:1016F00080E090E0262F30E0A901480F591F4830C4
:10170000510508F05EC1E62FE80FF0E0E35EFD4F03
:1017100040814D9301968C31910571F752C18A81B8
:10172000823039F0853009F04AC180E00E94BC2542
:1017300048C16B817C818D819E810E94442E0E94D4
:10174000901B3FC14C816B818A810E94581E26C12B
:101750002D813E813227232732274C816B818A815C
:101760000E94D61D2EC10E94FD1D2BC18A8183308F
:1017700009F025C12830B1F1293009F460C08B810E
:101780008230D1F070F4813009F01BC14C8128EC1B
:10179000429F412D11248091570320E0609158030E
:1017A0001DC08330B1F0843009F00BC18C8120E082
:1017B000409159036D8112C08C81811103C00E9438
:1017C000A325FFC00E94AF2560E08C810E945425B4
:1017D000F8C060E08C810E949524F3C090E00E94E4
:1017E000D024EFC08B818230E1F078F4813009F0B1
:1017F000E8C0809159032FEF829FC001112468EC4B
:1018000070E00E94162E6C83DCC08330A1F084301F
:1018100009F0D7C0809157038C83809158038D8342
:10182000D0C080915603982F937019F086958695B5
:1018300004C080E002C080915A038C83C2C048E09B
:1018400050E067E170E086E593E00E94D62D1092AB
:101850002303B7C080E152C082E08A8388E08B8393
:10186000B0C0EA80FB80FE24EF24FE24AC80B12CC3
:101870006801C70188509E4F9601201B310B2A1525
:101880003B0508F09EC0A8E0EA16A2E0FA0628F49C
:101890000E94C82DF601848303C0D60114961C92C1
:1018A000BFEFEB1AFB0AEFEFCE1ADE0AE2CFEA80B7
:1018B000FB80FE24EF24FE24AC80B12C6801C7011C
:1018C00088509E4F9601201B310B2A153B0508F0CE
:1018D00078C0F8E0EF16F2E0FF0628F4D60114967F
:1018E0006C910E94E62DBFEFEB1AFB0AEFEFCE1AC8
:1018F000DE0AE5CF0E94651D64C084E08A8361C072
:10190000EA80FB80FE24EF24FE24AC80B12C680129
:10191000C70188969601201B310B2A153B0508F05C
:1019200050C0F0ECEF16F1E0FF0630F40E94C82D35
:10193000D60114968C9302C0F6011482FFEFEF1AC1
:10194000FF0A2FEFC21AD20AE3CFEA80FB80FE24FF
:10195000EF24FE24AC80B12C6801C7018896960163
:10196000201B310B2A153B0560F5A0ECEA16A1E01F
:10197000FA0620F4F60164810E94E62DFFEFEF1ACB
:10198000FF0A2FEFC21AD20AE8CF41E08C81811101
:1019900001C040E06B818A810E94A21D9D831FC00F
:1019A0002D813E8132272327322741E08C8181110E
:1019B00001C040E06B818A810E94751D02C08FEFDB
:1019C000898340E250E0B80182E00E94B1195FCB08
:1019D00087E290E00E94C82D1B821C821D828E83AC
:1019E000F0CF2B30310508F037CD6CCD2B303105E1
:1019F00008F07ECDB3CDA8E0B0E0E1E0FDE00C94CE
:101A00004B2EFC018481882309F4DEC57F0121E08F
:101A1000408151816281738195810E949E2C8C014D
:101A2000F7019581992309F438C198013757203877
:101A3000310508F054C1003108F03FC18FEF93E049
:101A40000E94C82D811139C138EFA32EBB24B39455
:101A5000002379F0A114F4E0BF0609F42EC1C501FA
:101A60000E94C82D811101C001502FEFA21AB20AA5
:101A7000EFCFCE0101962C0188E0F20111928A95F8
:101A8000E9F72AE0322E85010F5F1F4FC5010E9442
:101A9000C82D89831A82882309F40FC1813009F087
:101AA00041C06501F2E0CF0ED11CC8010E94C82DD3
:101AB0008A83882309F401C19FEF980F933060F463
:101AC00023E0A20EB11CC6010E94C82D8B8388237F
:101AD00009F4F3C01C8229C0843031F54E0133E093
:101AE000830E911C02E010E056018FEFA81AB80A8D
:101AF000C6010E94C82DF40181934F01882309F487
:101B0000DCC08C3741F4E2E0F0E0EC0FFD1FE00FA9
:101B1000F11F10820AC00F5F1F4F650107301105CA
:101B200019F7CBC0580101C056018201F80120818C
:101B3000222309F4A8CF213009F053C081818130DC
:101B400081F46801F2E0CF0ED11CF8018281893363
:101B500019F460E570E002C060E070E00E94431894
:101B600015C0823049F46801F2E0CF0ED11CF801B3
:101B700082810E94CF170AC0833051F46801F2E0DD
:101B8000CF0ED11CF80182810E949C17860182C071
:101B9000843019F00F5F1F4F7DC0F80122810E5F66
:101BA0001F4F80E090E030E0205331092A303105AA
:101BB00068F4389EA001399E500D1124C901840F8C
:101BC000951F0F5F1F4FF8012081EDCF009709F49B
:101BD00061C0EFE9FFE03197F1F700C00000019725
:101BE000F5CFE22FF0E0E359FC4F2490822F869549
:101BF0008695869590E0FC01E35AFC4F649027702F
:101C0000712C022E02C0759467940A94E2F7F1E0F9
:101C10006F227724FC01E35BFC4F8490912C022E11
:101C200002C0959487940A94E2F731E083229924C4
:101C3000FC01E35CFC4FC490D12C02C0D594C79446
:101C40002A95E2F781E0C822DD246114710419F0BD
:101C500081EE0E94CF178114910419F086EE0E9444
:101C6000CF1760E070E0822D0E9443188114910428
:101C700019F086EE0E949C176114710419F081EE30
:101C80000E949C17C114D10429F060E070E08CE23E
:101C90000E9443180F5F1F4F49CFF801E851FC47DE
:101CA000E730F10508F082C104C106E221EE41EE01
:101CB0006AE17CE7C7010E94CD1B8091800287709A
:101CC00009F482C4F7018581882309F47DC48091D9
:101CD000010382FF79C482E00E94311675C4F801C5
:101CE000E851FC47E730F10508F4E3C01092F80230
:101CF000980130572332310508F003C184E090E0A9
:101D00000E94D02D9093010380930003F801E150CD
:101D1000F047E232F10520F4E559FF4F0C943E2ED6
:101D2000809100038160ACC0809101038860B4C0E1
:101D3000809100038260A4C08091000320C0809144
:101D4000000388609DC0809101031EC08091010343
:101D50008260A2C080910003806192C080910003E4
:101D600080628EC08091000380648AC00E948216C7
:101D700080910003806884C0809100038860846043
:101D80007FC0809101038260816086C080910003E2
:101D90008E7F76C080910103877F7EC08091000393
:101DA0008D7F6EC08091000320C080910003877FEB
:101DB00067C0809101031EC0809101038D7F6CC0BC
:101DC000809100038F7E5CC0809100038F7D58C09E
:101DD000809100038F7B54C00E9482168091000383
:101DE0008F774EC080910003877F8B7F49C08091A1
:101DF00001038D7F8E7F50C08091000382FB2227DC
:101E000020F991E0922790FB82F990FB83F938C08A
:101E100080910103982F909591708E7F892B90FB74
:101E200081F93AC08091000386FB222720F991E0D6
:101E3000922790FB86F924C00E94821680910003AD
:101E400087FB222720F991E0922790FB87F918C0A1
:101E500061E001C060E08EE090E00E94E62D1EC0CF
:101E60008091000384FB222720F991E0922790FBC8
:101E700084F906C080910003982F909590FB80F91B
:101E8000809300030BC08091010383FB222720F97C
:101E900091E0922790FB83F9809301036091000306
:101EA0007091010384E090E00E94042E0E9482164B
:101EB00004CFE357FF4F0C943E2E07E225EE45EE8C
:101EC0006BE17CE7F7CE06E221EE40EE68E17CE7CD
:101ED000F1CE07E225EE44EE69E17CE7EBCE06E2C7
:101EE00021EE42EE6CE17CE7E5CE07E225EE46EE20
:101EF0006DE17CE7DFCE08E221E045EE6EE17CE7B4
:101F0000D9CE80914C030631FCE71F0709F442C08B
:101F10008272F801E052F847EB30F10508F045C352
:101F2000EC56FF4F0C943E2E882329F00E948C25FE
:101F3000C4CE8823D9F30E949725BFCE882329F0E9
:101F40000E943E25BACE8823D9F30E944925B5CEFA
:101F5000882329F00E942225B0CE8823D9F30E943D
:101F60003025ABCE882329F00E940625A6CE8823F3
:101F7000D9F30E941425A1CE882329F00E94B82409
:101F80009CCE8823D9F30E94C42497CE81E00E947E
:101F9000BC2593CE8A7A91E009F490E090932502D3
:101FA000811112C089E20E94F11A0BC006312CE7A0
:101FB000120761F4809125028111F5C289E20E9425
:101FC000B21A0E94B82B79CE85E3EDCF80914C03F5
:101FD0008272F801E054F847ED30F10578F4E156EB
:101FE000FF4F0C943E2E0E94AF2502C00E94A325F5
:101FF000809123038160809323035FCE0737FCE742
:102000001F0711F481E005C008372CE7120749F4D7
:1020100082E00E94241643E062E081E00E94021602
:102020004CCE9801205E324520323105A8F4911142
:1020300016C00F7181E090E0FC0102C0EE0FFF1F9F
:102040000A95E2F78F016E2F83E090E00E94E62D63
:10205000802F0E947F1631CE992309F455C003309A
:10206000FCE71F07E9F1C0F401303CE71307F1F189
:1020700000F501159CE7190709F046C00E94821679
:102080003FEF84E39CE0315080409040E1F700C096
:1020900000000E94181A11CE0B35ECE71E0789F1DB
:1020A0000C35FCE71F0729F10A351C4769F581E06B
:1020B00029C08091FF02982F9095917090FB80F934
:1020C0008093FF02992319F08FEF93E002C08DEE09
:1020D00093E09F938F930E9401060F900F90EDCD98
:1020E0006FEF7FEF80E090E00E94042E0E94532D5E
:1020F000E4CD8091010382FB882780F991E0892754
:1021000001C080E00E944816F7018581008111819D
:10211000882349F0C8010E94E613D82E682FC80111
:102120000E94E51504C0C8010E94CC15D82EB80144
:102130008D2D0E94502A0E94702AD82E192FA82E69
:10214000F7010581C680C2949FE0C9228091800278
:10215000877001F10023F1F0812F807F803469F0D6
:1021600080E28D0D8830B0F0812F807E803229F49E
:10217000F1E0FD1578F4CC2069F08091010382FF35
:1021800009C082E00E943116809180028770BB24D2
:10219000B3948111B12C912E92948FE09822892DC5
:1021A00090E08C30910508F0D6C1FC01E455FF4F5A
:1021B0000C943E2E812F807F1F70882311F0129582
:1021C000107F0023B9F0112309F4B3C180E28D0D13
:1021D000883010F0A11006C090914C03192B109379
:1021E0004C0305C090918202192B109382020E9429
:1021F000B82B9FC18D2D0E949C17112309F4ABC1F0
:1022000080E28D0D883088F1AA2079F110959091A7
:1022100082021923109382022BC0812F807F1F70AE
:10222000803211F01295107F8D2DAA2029F021E027
:10223000A21609F44CC057C08091010382FD1BC057
:10224000002369F0112339F090914C03192B10935E
:102250004C030E94B82B80E00E94CF177CC180E025
:102260000E949C17112309F476C1812F0E94B12B83
:102270000E94B82B70C1002381F0CC20C1F131E065
:10228000C31269C190918102812F8923181709F423
:1022900062C1192B109381025EC1C1105CC1812FF4
:1022A0000E94B31680918102912F982329F0912FDB
:1022B000909589238093810220912602812F822389
:1022C00009F449C1109521232093260244C100231B
:1022D00029F085E08C1508F43EC109C094E09C15F6
:1022E00008F439C115C0002331F0C11022C1812F7B
:1022F0000E94BA1630C1CC2059F0893309F028C1A8
:10230000EFEFF7EE23E0E150F0402040E1F71EC18F
:10231000812F0E94B3161FC1812F869586958370E9
:1023200019F0813061F017C1002321F08D2D912F1C
:10233000937002C080E090E00E945E1B12C10023F7
:1023400021F08D2D912F937002C080E090E00E94CB
:10235000391B07C1602F8D2D0E94C41602C1812F29
:102360008370A9F50111FBC04D2D4295469547702C
:10237000440F440F8D2D8F7090E09C01042E01C0FE
:10238000220F0A94EAF7D4FE08C08FE090E001C063
:10239000880F4A95EAF7809501C080E0169516955A
:1023A0001370123069F088F490910E02113019F018
:1023B000822B892302C0922B892B0E947F16CFC0CB
:1023C000822B90910E028927F8CF822BF6CF002323
:1023D00019F0812F817001C08695882309F4BFC050
:1023E0004D2D429546954770440F440F8D2D8F70AB
:1023F00090E09C01042E01C0220F0A94EAF7D4FE5B
:1024000008C08FE090E001C0880F4A95EAF78095F8
:1024100001C080E0169516951370123059F078F4CB
:1024200090910F02113019F0822B892309C0922B51
:10243000892B06C0822B90910F02892701C0822B25
:102440000E94FF158CC01F70002339F0812F0E945D
:1024500073168D2D0E94BA1682C08D2D0E94B31660
:10246000812F0E9424167BC08D2D32EFA31681F19F
:102470003A1538F090EFA91659F0E1EFAE1619F1C0
:1024800054C0F3EFAF1659F124EFA216C1F04DC0BE
:10249000002381F034E03C1508F45DC01F7181E039
:1024A00090E0012E01C0880F0A94EAF790910F0284
:1024B00089271EC085E08C1508F44DC0EFCF8091B0
:1024C000010382FD1AC0002329F0812F8F7120C0E3
:1024D0000023D9F3812F8F710E9424163CC0002362
:1024E00051F01F7181E0012E01C0880F0A94EAF7B4
:1024F0000E94FF1530C080E0FBCF002361F0812FE8
:102500008F7198E0899F90011124236020938002AD
:102510000E94731620C081E00E943116E1E0EC15A4
:10252000D0F482E00E94311616C0002321F0CC20A6
:1025300061F28D2D91CECC2069F2893349F4FFEF01
:1025400027EE33E0F15020403040E1F700C00000BA
:102550008D2D0E949C1788EF890D843010F40E9405
:10256000831BBB20A9F08091800280FD11C0F70180
:1025700015828695869586950E947316C7010E94DE
:10258000FB0C809180028695869586950E94241684
:1025900020E0F701408151816281738184819581BE
:1025A0000E949E2C11C085E30ACD07373CE7130734
:1025B00011F481E006C008378CE7180709F031CD27
:1025C00082E00E94731627CD2896E2E10C94672ED4
:1025D00020917F029091460257E02917A9F030E040
:1025E000529FF001539FF00D1124E95BFD4F718163
:1025F000761306C07081781303C07581741306C00A
:102600002F5F3F4F2770E9CF80E0089581E0089564
:102610009B01782F777043E0969587954A95E1F76F
:10262000FC01EE0FFF1F8E0F9F1FF901E80FF91F2E
:1026300040E050E080E0219130E0072E02C0369566
:1026400027950A94E2F721703327042E01C0220F48
:102650000A94EAF7822B4F5F5F4F4330510559F7D9
:102660000895962F9770A1E001C0AA0F9A95EAF7F6
:1026700093E0769567959A95E1F7FB01EE0FFF1FC2
:102680006E0F7F1FFA01E60FF71F40E050E0682F42
:1026900070E090819B01042E02C0369527950A9424
:1026A000E2F72170219529272A23292721934F5FBB
:1026B0005F4F4330510569F7089590914C03809125
:1026C0008202892B909181029923E1F0892B9091CC
:1026D0000C01913041F49091000397FF04C09EE1FA
:1026E0002DE832E003C096E025E832E0F90120E071
:1026F000915028F031913323D9F32F5FF9CF211175
:1027000010928102089580917F029091460289176C
:1027100019F08F5F8770FBCF0895CF93DF9380917F
:10272000450282958F7009F04EC080914402882343
:1027300009F449C080917F024091460250914002C5
:1027400060913F02C0914102D091420277E084172C
:10275000D1F190E0789FF001799FF00D1124DF0115
:10276000A95BBD4F14962C911497222349F1119621
:102770002C911197251324C02C91261321C0159656
:102780002C91159721111CC012962D913C911397F5
:102790002C1B3D0B283C310598F4809145028F702D
:1027A000806180934502E35BFD4F80818F70806183
:1027B00080838FE392E00E94FB0C0E94831303C08E
:1027C00001968770C4CFDF91CF910895CF92DF92A9
:1027D000FF920F931F93CF93DF936C0100910F0231
:1027E00080910E02082BC3E0D0E010E0C8010C2E4F
:1027F00002C0959587950A94E2F780FD04C0219761
:10280000A8F7F12C09C0FC2EB6018C2F0E94502A8B
:102810000E94702A019799F38F2DDF91CF911F911C
:102820000F91FF90DF90CF900895CF93DF93EC014D
:102830000E94E613BE010E94502A0E94702ADF9176
:10284000CF910895FC0124812223D9F080819181C8
:102850000E94151492959F70963079F010F4925062
:1028600001C09A50923068F4803F69F018F4883EB5
:1028700040F409C0843F29F406C0883E20F0813F1F
:1028800011F080E0089581E00895A4E1B0E0EBE468
:10289000F4E10C94512E8C0186E0F801DE011F96C4
:1028A00001900D928A95E1F7F8018481E5809FE31C
:1028B000892E92E0992E90914302911120C0882395
:1028C00009F463C1EE2009F442C0C8010E94221439
:1028D000F82E8823E1F187E0F801D40101900D92F0
:1028E0008A95E1F780914302813031F480913F0273
:1028F000909140020E9415140E948D1348C1F80166
:10290000D080C180A280B380F09044022091410227
:1029100030914202FF2009F4E7C0A501421B530B8E
:10292000483C510508F09DC0882309F430C18091CE
:102930004502282F207F90914002222361F09C15B0
:1029400009F460C0C8010E942214811163C0C8014B
:102950000E94FB0C1AC19C1113C090913F029D1163
:102960000FC0E1100DC08F708061809345028FE32E
:1029700092E00E94FB0C80914502F801868303C11E
:10298000E1103AC040E06C2D8D2D0E94E81240E02D
:102990006C2D8D2D0E94E812E82E8111F4C0DF8687
:1029A000C88A8F8598890E941514292F22952F7027
:1029B000243020F49F70223028F009C02A502230A1
:1029C00080F014C0992349F0811107C013C09923E6
:1029D00021F0F8019681907F69F0805E883030F4B4
:1029E00009C0803F38F0815F833020F0C8010E9429
:1029F000FB0CEF2CFE2CCBC08091450281608093B4
:102A00004502C1C090913F029D119CCFE1109ACF29
:102A1000F80198C0EE2009F49ACF20914502822F48
:102A200082958F7090E002978CF080913F02909198
:102A3000400299878887BB86AA86809143028C874B
:102A40001D862E87CE0108960E94FB0C87E0F801B8
:102A5000AFE3B2E001900D928A95E1F70E948D13E9
:102A600094C090914502292F207F51F48FE392E08A
:102A70000E94FB0C87E0F40111928A95E9F783C06C
:102A8000882309F484C0809140028C110CC080918D
:102A90003F028D1108C0E11006C0F8019683C801FD
:102AA0000E94FB0C6AC0C8010E942214882309F40A
:102AB0004ECFEE2009F44BCF20914502822F829514
:102AC0008F7090E0029714F280913F029091400243
:102AD0009A838983BC82AB82809143028D831E825C
:102AE0002F83CE010196B0CFA21AB30AF8ECAF162D
:102AF000B10408F042C0882309F447C0FE2CEE2040
:102B000009F425CF809140028C1129C080913F02A9
:102B10008D1125C09091450290FD18C0892F829596
:102B20008F70282F30E02115310581F0F801968350
:102B30002F30310541F08F5F982F9295907F8681DD
:102B40008F70892B8683C8010E94FB0C87E0F801F7
:102B5000AFE3B2E001900D928A95E1F718C0C80189
:102B60000E942214811172CF80914502816080936E
:102B70004502C8010E94FB0C0AC087E0F4011192D3
:102B80008A95E9F704C0F12C02C0FF24F3948F2D3D
:102B90006496ECE00C946D2E292F983058F4873011
:102BA00048F490E06AE272E037E0239F800D911DC7
:102BB000112406C02C5F223030F467E272E090E00E
:102BC0000E940813089580E00895282F862F9830DA
:102BD00060F4273050F4622F70E027E0929F600D80
:102BE000711D11244AE252E007C09C5F923030F41C
:102BF000622F70E047E252E00E9431130895809303
:102C00000F02089590910F0221E030E0F90101C018
:102C1000EE0F8A95EAF7D90102C0AA0FBB1F6A9589
:102C2000E2F7BD016E2B01C0220F4A95EAF7892F0A
:102C30008623681303C0892F822B03C02095822F1F
:102C400089230E94FF15089521E030E001C0220F82
:102C50008A95EAF7209580910F0282230E94FF1542
:102C60000895909180028095892380938002282F77
:102C7000277069F4981759F09091010392FF07C0EB
:102C80008695869586950E94241610928002089556
:102C9000CF939091010392FB222720F9281709F185
:102CA000C82F892FC0FB82F9809301036091000334
:102CB0007091010384E090E00E94042E82E00E9463
:102CC00031168091FF0280FF0CC01F92CF9380E1EC
:102CD00094E09F938F930E9401060F900F900F90A6
:102CE0000F90CF91089521E030E001C0220F8A9526
:102CF000EAF780910F02822B0E94FF1508958093BE
:102D00000E02089510924C0380910C01813041F421
:102D10008091000387FF04C08EE1EDE8F2E003C07C
:102D200086E0E5E8F2E0DF011D928A95E9F780E0B0
:102D300090E00E945E1B80E090E00E94391B1092A0
:102D400082020E94B82BE0EFF2E086E0DF011D92E4
:102D50008A95E9F71092EB021092E9021092EA02CA
:102D60000E94511C0895882321F00E94B12B0E94DB
:102D7000B82B0895882339F090914C03892B8093C8
:102D80004C030E94B82B0895662309F45CC08D3C67
:102D900021F40E94371D819504C08E3C29F40E94C5
:102DA000371D8093F302C5C08F3C21F40E94371D6C
:102DB000819504C0803D29F40E94371D8093F20262
:102DC000B8C0893D19F40E94151D05C08A3D31F433
:102DD0000E94151D81958093F402ABC08B3D21F4B8
:102DE0000E94151D819504C08C3D29F40E94151D7B
:102DF0008093F5029EC09FE2980F983078F421E00E
:102E000030E0A90102C0440F551F9A95E2F7CA01AC
:102E10009091F102892B8093F1028BC08D3D21F4BA
:102E20008091EA0281600CC08E3D21F48091EA021B
:102E3000826006C08F3D09F07CC08091EA02846008
:102E40008093EA0276C08D3C39F49091F30297FFAB
:102E500035C01092F30259C08E3C29F49091F302D0
:102E60001916BCF32BC09091F2028F3C29F497FF06
:102E700025C01092F20249C0803D19F41916CCF316
:102E80001DC09091F402893D29F41916BCF41092EA
:102E9000F4023BC08A3D19F497FF10C0F8CF8B3D78
:102EA00039F49091F50297FF09C01092F5022DC0F8
:102EB0008C3D21F49091F5021916BCF39FE2980F16
:102EC000983080F421E030E0A90102C0440F551F82
:102ED0009A95E2F7CA0180959091F1028923809337
:102EE000F10213C08D3D21F48091EA028E7F0BC068
:102EF0008E3D21F48091EA028D7F05C08F3D29F43B
:102F00008091EA028B7F8093EA028091F202811124
:102F100006C08091F302811102C01092EB028091F1
:102F2000F402811106C08091F502811102C0109255
:102F3000E9020E94511C0895882381F19CEF980FAB
:102F4000913A18F40E94B21A0DC090E2980F98308E
:102F500060F4877091E001C0990F8A95EAF7892F94
:102F60000E94B12B0E94B82B08959BE5980F9330D7
:102F700028F480E090E00E945E1B089598E5980F89
:102F80009B3128F480E090E00E94391B089593E380
:102F9000980F933118F460E00E94C4160895CF93FF
:102FA000882309F46EC0C82F8CEF8C0F813AA0F5EE
:102FB00080910C018130E1F48091000387FF18C0FB
:102FC000EC2FE695E695E695F0E0E557FD4F82811A
:102FD000282F30E04C2F477081E090E002C0880F2E
:102FE000991F4A95E2F782239323892B61F410C03D
:102FF000E5E8F2E08BE892E02191C21721F08E170C
:103000009F07D1F705C08C2F0E94B21A0E94B82BDF
:103010008C2F0E94F11A10C080E28C0F883078F457
:10302000C77081E090E001C0880FCA95EAF79091DF
:103030004C03892B80934C030E94B82B22C0EBE5F4
:10304000EC0FE33040F4F0E0E35AFE4F808190E073
:103050000E945E1B16C0E8E5EC0FEB3150F4F0E087
:10306000EE0FFF1FE05AFE4F808191810E94391BB5
:1030700008C083E38C0F833120F461E08C2F0E9421
:10308000C416CF9108951F93CF93DF93182FEB01B0
:103090000E94CF17209741F08FE99FE00197F1F749
:1030A00000C000002197F6CF812F0E949C17DF916E
:1030B000CF911F91089580910B010895FC01EE0FAF
:1030C000FF1F8E0F9F1FFC01ED54FD4F6183408356
:1030D00022830895E3EBF2E0818360834283339699
:1030E00092E0E93EF907C1F70895509A08959FB715
:1030F000F894109208039FBF90911503943009F043
:1031000057C09091E9009F703091EC00232F2170FF
:1031100030FD20E8922B25E02093E9002091EB0080
:1031200020FF43C02091EE0027FF3FC020910703FE
:10313000222321F02091E80025FF37C010920703D9
:1031400026E03091E80035FD15C03091150334308C
:1031500061F53091EB0035FD28C0215021F481E06C
:103160008093070322C0EFE9FFE03197F1F700C039
:103170000000E7CF8093F1008091E80085FD0AC050
:103180008091E80080FFFCCF8091E8008E778093EB
:10319000E80006C08FB7F89421E0209308038FBFA2
:1031A0009F709093E90080E008959F709093E900EC
:1031B0008FEF08958BB18E7F9BB191602FB7F894FC
:1031C000E3EBF2E032E0E93EF30789F0319148E0C9
:1031D0009BB9000000C037FF8BB9330F000000C05F
:1031E00000C000C08BB900C04A9591F7EBCF2FBF4C
:1031F0008FE594E00197F1F700C0000008958091F9
:10320000170387FF11C08091E80082FD05C08091FF
:1032100015038111F8CF11C08091E8008B770BC0A6
:1032200080911503882349F08091E80080FFF8CF52
:103230008091E8008E778093E8000895982F97306A
:1032400068F59093E900981739F07091EC0020919F
:10325000ED005091F00003C0242F762F50E021FDA7
:1032600002C09F5FECCF3091EB003E7F3093EB00CC
:103270003091ED003D7F3093ED003091EB003160F7
:103280003093EB007093EC002093ED005093F0002E
:103290002091EE0027FDE5CF80E008958F708093A8
:1032A000E90081E0089520911D0330911E03261747
:1032B000370748F06115710539F42091E8002E7741
:1032C0002093E80001C0B901FC0120E061157105FF
:1032D00079F1809115038823F1F18530F1F1809126
:1032E000E80083FD3CC08091E80082FD2EC0809103
:1032F000E80080FFEBCF2091F3008091F20090E096
:10330000922B6115710551F08830910538F42191A7
:103310002093F100615071090196F3CF21E00897E5
:1033200009F020E08091E8008E778093E800CECF0E
:103330002111CFCF0AC080911503882361F0853019
:1033400061F08091E80083FD0AC08091E80082FF6F
:10335000F2CF80E0089582E0089583E0089581E04F
:1033600008950F931F93CF93DF938B01EA01909100
:103370001503943079F58F708093E9008FEF909169
:10338000E800815095FD06C095ED9A95F1F7000093
:103390008111F5CF8091E80085FF1CC00E94B82301
:1033A000882361F08091E8008E778093E80012C056
:1033B000F80181918F018093F1002197209791F37B
:1033C0008091E80085FDF4CF8091E8008E778093AE
:1033D000E800E4CFDF91CF911F910F91089543E072
:1033E00050E0BC0184E00E94B119089546E050E02D
:1033F000BC0184E00E94B119089540E250E0BC0194
:1034000084E00E94B1190895CF93DF93EC0148E066
:1034100050E0BC0181E00E94B11988E0FE01ABE000
:10342000B3E001900D928A95E1F7DF91CF91089575
:1034300081E08093E00080E28093D8001092C90080
:103440008FE19EE40197F1F700C0000087E090EB68
:10345000DC0180935E0390935F03A0936003B093BD
:1034600061039CE088E10FB6F894A8958093600012
:103470000FBE90936000FFCF78941F920F920FB60B
:103480000F9211248F939F93AF93BF938091030367
:1034900090910403A0910503B09106030196A11D2C
:1034A000B11D8093030390930403A0930503B0938D
:1034B0000603BF91AF919F918F910F900FBE0F9018
:1034C0001F9018959C014FB7F89480910303909139
:1034D0000403A0910503B09106034FBF821B930B19
:1034E00008952FB7F89460910303709104038091BD
:1034F0000503909106032FBF08952FB7F89480918C
:10350000030390910403A0910503B09106032FBF1C
:1035100008951F920F920FB60F9211248F939F93CD
:10352000AF93BF9380910203811113C08091030375
:1035300090910403A0910503B09106034196A11D4B
:10354000B11D8093030390930403A0930503B093EC
:103550000603BF91AF919F918F910F900FBE0F9077
:103560001F90189590910C01913021F490910003D7
:1035700097FD03C0E3E8F2E02EC0E82FE695E6955C
:10358000E695EE3190F4F0E0E557FD4F877021E0CD
:1035900030E0A90102C0440F551F8A95E2F7CA0125
:1035A000809592818923828308959091FF0290FFF4
:1035B00017C01F928F938DE596E09F938F930E9483
:1035C00001060F900F900F900F900895319652E0E2
:1035D000E938F50729F092818913F8CF1282F6CFE6
:1035E000089590910C01913059F59091000397FF47
:1035F00027C0E82FE695E695E695EE3180F4F0E0F9
:10360000E557FD4F877021E030E0A90102C0440F6B
:10361000551F8A95E2F7CA019281892B27C09091A4
:10362000FF0290FF25C01F928F938FE396E09F9338
:103630008F930E9401060F900F900F900F900895A6
:10364000A5E8B2E0EFEF90E02D91821789F0EF3F0F
:1036500019F4211101C0E92F9F5F9630A9F7EF3FC0
:1036600039F00E2E000CFF0BED57FD4F82830895AD
:103670000895A3E0B0E0EFE3FBE10C945B2E209112
:10368000FD023091FE0228173907A1F09093FE0247
:103690008093FD02E091FB02F091FC02309751F023
:1036A00024E029839B838A830084F185E02DCE0169
:1036B000019609952396E2E00C94772EA3E0B0E002
:1036C000E4E6FBE10C945B2E2091F9023091FA02C2
:1036D00028173907A1F09093FA028093F902E0913C
:1036E000FB02F091FC02309751F023E029839B8389
:1036F0008A830084F185E02DCE01019609952396F9
:10370000E2E00C94772EE091FB02F091FC023097FE
:1037100029F00190F081E02D0995089580E0089549
:1037200087E290E00E94E62D0895CF93C82F811183
:1037300002C06FEF01C065E284E290E00E94E62DD6
:10374000C11102C06FEF01C061E085E290E00E940C
:10375000E62DC11102C06FEF01C064E186E290E086
:103760000E94E62DCF91089584E290E00E94C82D3A
:10377000853281F485E290E00E94C82D813051F4B9
:1037800086E290E00E94C82D91E0843109F090E03B
:10379000892F01C080E0817008950F931F93CF930C
:1037A000DF93C42FD22FFC0185818823B1F0409391
:1037B000F8020E947D1A9093F7028093F60280E24D
:1037C0008C0F883008F068C0C77081E001C0880F96
:1037D000CA95EAF70E94BA165FC08091F8024813B2
:1037E0003DC08091F6029091F7020E94621A883CD7
:1037F0009105A0F510E21D0FCD17E9F080E28C0FC6
:10380000883040F4C77081E001C0880FCA95EAF79C
:103810000E94B316183078F581E09D2F977001C093
:10382000880F9A95EAF70E94BA16093351F560E5B8
:1038300070E089E329C0093319F460E570E002C043
:1038400060E070E0802F0E944318183028F5D77090
:1038500081E001C0880FDA95EAF70AC080E28C0F98
:103860008830D0F4C77081E001C0880FCA95EAF7AC
:103870000E94B31611C0093351F460E570E089E38A
:1038800009C060E070E0802F0E944318E0CF60E044
:1038900070E0802F0E944318DF91CF911F910F910C
:1038A00008958091FF0283FF96C08CE196E09F937C
:1038B0008F930E9401068091F1021F928F9387E1FE
:1038C00096E09F938F930E94010685E196E09F9377
:1038D0008F930E9401068091F202282F082E000C7F
:1038E000330B3F938F9382E196E09F938F930E94D7
:1038F000010680E196E09F938F930E9401068091DC
:10390000F302282F082E000C330B3F938F938DE08A
:1039100096E09F938F930E9401068BE096E09F9321
:103920008F930E9401068091F402282F082E000C2C
:10393000330B3F938F9388E096E09F938F930E9481
:10394000010686E096E09F938F930E940106809186
:10395000F502282F082E000C330B3F938F9383E042
:1039600096E09F938F930E94010680E096E09F93DC
:103970008F930E9401068DB79EB780960FB6F8947C
:103980009EBF0FBE8DBF8091EB021F928F938DEF74
:1039900095E09F938F930E9401068BEF95E09F9394
:1039A0008F930E9401068091EA021F928F9388EF05
:1039B00095E09F938F930E94010685EF95E09F937A
:1039C0008F930E9401068DB79EB70C960FB6F894A0
:1039D0009EBF0FBE8DBF0E947D1A2091F202211161
:1039E00004C02091F302222321F09093EF028093F0
:1039F000EE022091F402211104C02091F50222234D
:103A000021F09093ED028093EC02E091FB02F091A3
:103A1000FC02309749F082E08093F0020680F78143
:103A2000E02D80EF92E0099508958091EA0280FDF3
:103A300016C081FD16C082FD18C08091E90288235E
:103A400091F0883290F428E0829FC001112468E24E
:103A500070E00E942A2E862F672B29F007C082E093
:103A6000089584E0089581E0089588E008958091A4
:103A7000EA0280FD14C081FD14C082FD16C0809151
:103A8000EB02882381F08E3180F420E5829FC00113
:103A900011246EE170E00E942A2E862F089584E1A1
:103AA000089588E2089588E0089580E50895282F14
:103AB00035EB2303C001112497FF03C080589109FF
:103AC00002C080589F4F892F0895CF93DF93C8EF8E
:103AD000D1E060E0CE010E94E62D2196C11584E080
:103AE000D807B9F7DF91CF9108950F931F93CF9324
:103AF000DF93843010F5611120C094E0899FE001CC
:103B00001124C851DE4F411103C082E090E002C091
:103B100080E090E0632F022F142F8C0F9D1F0E94D6
:103B2000E62D111103C083E090E002C081E090E037
:103B3000602F8C0F9D1F0E94E62DDF91CF911F916A
:103B40000F910895FF920F931F93CF93DF938430CB
:103B500030F5611124C024E0829F800111240851B6
:103B60001E4F411103C082E090E002C080E090E06F
:103B7000F42E800F911F0E94C82D90E0D82FCC27E3
:103B8000F11003C083E090E002C081E090E0800F7C
:103B9000911F0E94C82D9E01282BC90102C080E000
:103BA00090E0CDB7DEB7E5E00C94742E1F93CF9371
:103BB000DF93962F8430E8F46830D8F44730C8F4A7
:103BC000632F122FC42FD0E0CC0FDD1F2EE0929F69
:103BD000C00DD11D112490E7899FC00DD11D112466
:103BE000CE0188960E94E62D612FCE0189960E9413
:103BF000E62DDF91CF911F910895A0E0B0E0E3E0C2
:103C0000FEE10C94512E05EE15E0C12CD12C912C27
:103C1000812CE12CF12CC0E0D0E05601AE0CBF1C91
:103C2000FE01EE0FFF1FEA0DFB1DEB5DFB4F259123
:103C300034914C2F682D892D0E94D61D2196C730B6
:103C4000D10571F78EE0E80EF11C839488E08812AC
:103C5000E2CFF8012591349141E060E0892D0E9486
:103C6000751DF80132962591349140E060E0892D70
:103C70000E94751D0C5F1F4F939480E7C80ED11CE6
:103C800084E09812C5CFCDB7DEB7ECE00C946D2E72
:103C900080E00E94951B60E070E0CB010E94901BC9
:103CA0000E94FD1D0E94651D81E00E94951B0895E4
:103CB0000F931F93CF93DF93843008F56830F8F4A7
:103CC0004730E8F4C42FD0E0CC0FDD1F2EE0629F18
:103CD000C00DD11D112430E7839FC00DD11D1124CB
:103CE000CE0188960E94C82D90E0182F0027CE01A3
:103CF00089960E94C82D9801282BC90102C080E036
:103D000090E0DF91CF911F910F910895611102C052
:103D100025E301C026E383B190E02F7002C09595A2
:103D200087952A95E2F781700895611102C085E3B5
:103D300001C086E334B1282F2F7081E090E001C0EC
:103D4000880F2A95EAF7982F9095932394B995B107
:103D5000892B85B908959091AD02E92FF0E040914B
:103D6000AE0250E09F012F5F3F4F23703327421771
:103D70005307A1F0E155FD4F8F7720812078822BEA
:103D800060FB87F980839F5F93709093AD02809171
:103D9000AB028F5F8093AB0281E0089580E00895CD
:103DA000AAE2B0E0E6EDFEE10C945A2EE7E1F3E082
:103DB0008091F100819343E0EF31F407C9F78091DE
:103DC0001803833009F463C030F4813071F082301D
:103DD00009F4A2C0B9C08A3009F48EC08B3009F44E
:103DE0006EC0893009F0B0C020C080911703813ABD
:103DF00009F0AAC08091E800877F8093E800809155
:103E00001B0390911C03892B21F468E08BE093E065
:103E100003C060E080E090E070E00E945319809160
:103E2000E8008B778093E8008FC080911703813280
:103E300009F08AC080911B0390911C03009719F030
:103E4000029709F081C08091E800877F8093E800A5
:103E50008091E80082FD05C0809115038111F8CFA3
:103E600073C02091F3008091F20090E0922B0297B2
:103E700031F48091F100813011F0863021F480918D
